:06000000022FFD02035B6C
:03000B0002008070
:0300130002036E77
:03001B000200B030
:03002B00020329A4
:03005B0002037D20
:030073000203483D
:20008000C0D075D01018B8CF0408208507B285868AD0D03253A4DFD285C2A98F8E7589AAAE
:2000A000C289C28B758A00D2A8D2AAC228D0D032C2A8C28E85578BC0D075D008C0E0C0F0A9
:2000C000C2CAA9CEAACFD2CAC3E99558F9EA95597049C3E9955A4043955A503FB8103C78CD
:2000E00000A9567D00E2FEC39DC399402E99EC33FC08E2FDC39EC399402199EC33FC08E223
:20010000FEC39DC399401499EC33FC08E2FDC39EC399400799EC33FC088002806AE2FEC367
:200120009DC399406299EB33FB08E2FDC39EC399405599EB33FB08E2FEC39DC399404899C2
:20014000EB33FB08E2FDC39EC399403B99EB33FB08E2FEC39DC399402E99EB33FB08E2FD0A
:20016000C39EC399402199EB33FB08E2FEC39DC399401499EB33FB08E2FDC39EC39940071A
:2001800099EB33FB08801E0530E53070021530C3E5309432400AD225755B00755C0061190C
:2001A00075310A6119E2FEC39DC39940DA99EA33FA08E2FDC39EC39940CD99EA33FA08E264
:2001C000FEC39DC39940C099EA33FA08E2FDC39EC39940B399EA33FA08EBC46B6C6A30271F
:2001E00001F4540F70A1C3EBF4FA9460FBECF4540F9400FC5018EA7C007B00600CC313505D
:2002000007B55B05055C8006E4F55B755C0030221BC3EB94D0F5F0EC94074003ABF0FC30E1
:200220002101B39226C3EB33FBEC33FCEB54F04CC475F00584FAEC13FCEB132AFBEC3400D5
:20024000FC30E3047BFF7C07201C27301124EC700C798187F0C3EB95F05002ABF0E5376051
:200260001175F028A42BFBEC3400FC30E3047BFF7C07EB54F84CC423F97007EB7004D225B6
:200280008005753200C225E53060021530C3E54CFD954D4002AD4DC3ED995008ED75F00885
:2002A000A4FBACF08CF0EBA2F013A2F113F4F9EC0303F45401FA30291CEBF4540324C0F8A8
:2002C000E623F630E00FE92401F97009EA3400FA30E1021A19C3E9941EFBEA9400FC5005FA
:2002E000E4FBFC800DC3EB954FEC95504004AB4FAC5089E98AEA8BFB8CFC75310A302719E5
:20030000302816758E017589A2D28543A420780085638AC28DD2A980097800758A00D2A83F
:20032000D2AAD0F0D0E0D0D032C0E0C2CF053BD223E5317004D22580021531302507E532DD
:200340000460020532D0E032C2AF53E67F53917F7592FA7593FFC218D2AF32C0E0E58A8569
:20036000578BC0D075D008F208D0D0D0E032C2AAD28EC2CA85CE5885CF59D2CA32327A0018
:200380007901801E7A00790580187A00790A80127A007964800C7A0079C880067A0079FA15
:2003A0008000090A8009781874FFD5E0FDD8F9D9F5DAF3227A427B3580247A2D7B4D801EC1
:2003C0007A267B5C80187A197B8C80127A147BAF800C7A427B1E80067A2D7B2C8000E553BD
:2003E0007001227902E4C292D5E0FDC293D5E0FDD293D5E0FDD292D5E0FDE920E002C29193
:2004000030E002C295E553D5E0FDE920E002D29130E002D2957496D5E0FDD9C9EA78C8D862
:20042000FED5E0F9DBBDC2922271B471BA71C02271D871B42271C071BA71B4227999875340
:20044000B8010471B48017B8020471BA8010B8030471C08009B8040471C6800271CC79986A
:20046000875322903070E493F4601D7C3E903074E493A3FB6012E493FA600471DE8006EB5E
:20048000F97A0071A2A3DCE82278A5E6F954037000E9540C7000E954307000E954C0700087
:2004A00022D291D293D295C290C292C29475D5FF22201E2E78FF201026E53A6022E5426023
:2004C0001E74FF301102747F8542F084853AF0A4F8C5F0600278FFC3E8954E5002A84E88E3
:2004E0004D22C3E54194A0E5429400E54D5003148001046002F54D22102301220566E566C5
:200500005403B4012CE551604F7552FFE5BE6048E5BDC3955140417552C89404403A755279
:2005200096940440337552649404402C7552328027B4021EE5516020C3E54C95526019402D
:2005400008E54C6013154C800FE54C046002054C8006B4030375E895302438E566541FB4E7
:200560000412E5BE7003E48004E5BD9414F564756502801FB408087564887565088014B47A
:200580000C087564AA75650A8009B410067564CC75650C227541007542F022C2AFC2CAA8BC
:2005A000CEA9CFAA3B30CF010AD2CAD2AFC3EA13FAE913F9E813F8201014C3E8953C883CC3
:2005C000F8E9953D893D547FF9301E36C1B5AB3CAC3DAD3E883C893D8A3EC3E89BE99CEA1A
:2005E0009D547F60087541FF7542FFC184AE3FAF408B3F8C40C3E89EF8E99FF9AA41AB4267
:200600008011AA41AB42C3EB9404404894044013201126C3EB13FDEA13FCC3ED13FDEC13EB
:20062000FC804AEBC423FCEAC423541F4CFC7D00C3E913F9E813F88034EBC423FC541FFD80
:20064000EC54E0FCEAC423541F4CFCC3E913F9E813F88019EBC4FCEAC4540F4CFC7D00C36A
:20066000E913F9E813F8C3E913F9E813F8C3EA9CFAEB9DFBEA28F541EB39F5425006754172
:20068000FF7542FFC3E54294025002D21EE542C4FA540FFBEA54F0FAE541C4540F4AFAC324
:2006A000EA9402FAEB9400FB40057048EA70457A017B00803FAA41AB42EBC4FCEAC4540F61
:2006C0004CFCC3EA9CFAEB9400FBE80303543F2AFAEB3400FB8A418B42C394024002C21E43
:2006E000EBC4FE7B00EAC4540F4EC39402FA400270027A01202806301808120ABF3018022E
:2007000080FB854892854993D21843E6807892E6FFC3E49AF8E49BF9C3E833F8E933F92060
:200720001E7F3010047F038015C3E5389482400E0F941E40010FC3EF940640027F05E8FA78
:20074000E9FBD3E913FDE813FC8C468D4788488949C3EF9403602BEF20E00CE82CF8E93DA9
:20076000F9ECFAEDFB800BE8D338F8E939F97AFF7BFFC3EF9403400A8A4A8B4B8844894557
:200780008050884A894B8A448B45301045754AF0754BFF7546F07547FF7548F07549FF8002
:2007A00031E8FAD313FC8C468848C3EF9403601EEF20E007E82CF8ECFA8007E8282401F83F
:2007C0007AFFC3EF940340068A4A88448004884A8A44202806301808120ABF30180280FB0F
:2007E000753502D21843E68030112DA841A942C3E913F9E813F8301004E92440F9C2AF537F
:20080000E67F759100C3E498F594E499F595759104D21843E680D2AF2275F000301D0E7529
:20082000F040800975F040301D0375F000D2197543007A027B02201E1D301102C219301050
:20084000067A367B36800F7B28E542700104FAC3942840027A28201811E543600D301003E5
:20086000D53504D21A80671207E30543E59B5440B5F00DE53460BB2019B8DADAC21A804E0A
:2008800020100B2019110AC3EA9B40CA80A40AC3EA9B40011A80BFC21953E67F759100309E
:2008A0001E117594007595F0759104D21843E680020832E5427EFFC3334009C3334005C34C
:2008C000334001FEC3E49E759400F59580DAC2AF53E67F854492854593759100854A9485A5
:2008E0004B95759104D21843E680D2AF201013301A1220110F201D0C201909158115810262
:20090000120B053422E53875F007A430190105F0A2F013A2F113A2F213F538C394785003B2
:20092000753878C3E53895394009D291D293D29575D5FF20280530180751BF30180280FBB2
:20094000854692854793D21843E6802220120FC2AFC292D29075D5CFD2AF759F1022C2AF6D
:20096000C292D29475D5FCD2AF759F102220120FC2AFD29575D5F3D290D2AF759F1122C26E
:20098000AFD29175D5F3D294D2AF759F122220120FC2AFC290D29475D5F3D2AF759F122269
:2009A000C2AFC294D29075D5F3D2AF759F112220120FC2AFD29375D5FCD294D2AF759F10A1
:2009C00022C2AFD29375D5CFD290D2AF759F102220120FC2AFC294D29275D5FCD2AF759F96
:2009E0001122C2AFC290D29275D5CFD2AF759F122220120FC2AFD29175D5CFD292D2AF7533
:200A00009F1222C2AFD29575D5FCD292D2AF759F11227432A28540032085F750033085F213
:200A2000D5E0F3922722E55B700122F8C39406500FC2AF1204A112043C120396D2AF80780E
:200A4000C3E55C94064077B80704C221806AB80804D2218063B80904C222805CB80A04D2FA
:200A6000228055B80D0A75640075650ED2248048B80E0A7564FF75650EC224803BB8140A2A
:200A80007988E714A2E09221802EB8150B7988E714A2E0B392218020B80C1DE4A22192E021
:200AA000A22292E1047988F77554A57555F1B128755400755500D2AF755B00755C0022C06A
:200AC000D075D010BE002DE5657022C2AF854126854227D2AFE526A23813F9A2391329F561
:200AE00026E52703C2E7F903C2E739F5270E201803D0D022BE0124E5657010E527705DE5A8
:200B000026701175270F7526FF80098564268565277565000E201803D0D022BE0215E5267B
:200B2000C465266527F478D0A65D71D90E201803D0D022BE030BE52671D90E201803D0D03C
:200B400022BE040CE526C471D90E201803D0D022E52771D9087E00D0D0D2282220E71620AC
:200B6000E61D20E52720E43420E34120E25020E15CE5266114A23733F52675270F6114A2B2
:200B80003733A23633F52675270D6114A23733A23633A23533F52675270B6114E52654F000
:200BA000C23C4527C4F5267527096114E526A23813A23913A23A13F5267527076114E526BF
:200BC000A23813A23913F5267527056114E526A23813F5267527036114540F23900BE0736E
:200BE0008100810A811781288132813F8149815D816A817E8185819681A081B781C181D595
:200C000008A65F08A65D08A65D2208A65D08A65E08A65D08A65D2286F0E55EB5F002E55F9C
:200C2000F608A65F08A65D2208A65D08A65F08A65D2208A65E08A65D08A65D08A65D2208E8
:200C4000A65E08A65E08A65D2286F0E55EB5F002E55FF608A65D08A65E08A65D2208A65D6E
:200C600008A65D08A65E08A65D2286F0E55EB5F002E55FF608A65E08A65D08A65D2208A6A4
:200C80005F08A65E2286F0E55EB5F002E55FF608A65E08A65E2208A65D08A65E08A65E22AE
:200CA00086F0E55EB5F002E55FF608A65D08A65D08A65D08A65D2208A65E08A65D08A65E29
:200CC0002286F0E55EB5F002E55FF608A65D08A65D08A65E2208A65D08A65D08A65D08A645
:200CE0005E2290300D7820B165E520B4550AA3B165E520B4AA0280127554A57555F1B1EC6B
:200D0000B128755400755500801D90300378807B0AB165A308DBFA90300F788C7B1AB16576
:200D2000A308DBFA90302922C2AFB1A8B1CAB1859030007400B16AA37412B16AA374CCB186
:200D40006A90300378807B0AB169A308DBFA90300F788C7B1AB169A308DBFAB1BBB1DDB1A2
:200D60009990302922E493F622E6438F01538FFDFFC3E58394F0400122EF8554B78555B787
:200D8000F0538FFE22438F02438F018554B78555B790300DF0538FFC2290300D7455B16A2B
:200DA00090300E74AAB16A227A3079D07820903040B165E520F709A3DAF7227A3079D0904B
:200DC0003040E7B16A09A3DAF9227A8C79007820903070B165E520F309A3DAF7227A8C798D
:200DE00000903070E3B16A09A3DAF922788076FF0876330876010876010876190876FF08EC
:200E000076090876300876010876FF08080876FF0876FF0876FF0876FF0876FF0876FF08A3
:200E200076040876FF0876FF0876FF0876FF0876FF0876280876500876040876FF087602D4
:200E40000876FF0876FF0876FF0876070876FF0876FF0876FF087600087600227888E61407
:200E6000A2E19222A2E092217884745096500276507886740D965002760D863A789CE6757F
:200E800039FFB402037539A0B4030375398275510078A0E6F8600674532409D8FCF5517881
:200EA000988653788DE623F95401F550E954FEF54FB6FF03754FFF7883E624FF922978C02F
:200EC0007600087611087655087677227554007555007597DE7597AD7581B075EF0675A9BF
:200EE000001204A17580FF75F1E175A4007580FF75D4FF75902A75F23F75A53F75902A75D9
:200F0000D5FF75A60175A72075F30175A70075E34075E2021204A1E4F8F6D8FDB1EC91E2C1
:200F2000D15CC2AF120390120463120489120390C2AF7554007555001204A175A91375A7A9
:200F40001075C10075A700780979007A0030850CDAFBD9F9D8F712043002F000302A0E12D2
:200F6000042912039C12039C12039CC22A758851758E017589AA758C00758D0075C8047592
:200F8000910475D84075D90875F781759E0775960375DB4275DA42759B80759D00759D40AD
:200FA00075AF1875B90A75DF2F75BB1075E88575B22012037E511275E4D530270375E45D9D
:200FC000C228C22475A82D75E68075B803D2AF758E0C755780755610755A50755DF7755E7A
:200FE000E7755FD67563E17560EB7561CA7562A975300A120390E530602B7557C075560874
:20100000755A28755DFF755EF7755FEF7563E17560FB7561EB7562DA75300A120390E53017
:201020006003020F30C0D075D010AF8ED0D0D22A753700C2AF1203D2D2AFC3E532940A4011
:20104000F9C2AF1203D8D2AFE4F541F542F55BF55CF533F53BC3E53B945E4033753B000571
:2010600033789AE67814146012782814600D786414600878C8146003753300C3E5339840A8
:201080000E15337804C2AF1204A112043CD2AF202806120ABF1204F830250CE53170030260
:2010A0000F30120A2680AE1203902025A8C2AF1204A1D2AFE4F522F523F53812037E756599
:2010C00000C2AF7984874E854E4C854E4D854E5275A71075C11075A70075A903C3E5573388
:2010E000F557C3E55A33F55AC3E55633F556E55DC560F55DE55EC561F55EE55FC562F55F70
:2011000075633CD2AFA2219212302204A2269212D210D21175340075360C1209D01209F1F5
:2011200012059412059B12059412059B12059412082412090512094C12059B12081912048A
:20114000B112090512096D12059B12082412090512098E12059B1208191209051209AF129C
:20116000059B1208241209051209D012059B1208191209051209F112059B1204F83011353F
:2011800030101A854E4CC3E5349418500530259F807EC210754CFF754DFF7552FF201D159C
:2011A000E53614600AF5363025852022828061C211D21C212F753700D21B30251320220C8C
:2011C00079A4E76007C3E53294035044E5316040202209C3E54294F05036212F201D1220EB
:2011E000120520260580EC2026E9D21D854E4C2156854E4CC3E5429420400EC21DA2269229
:2012000012D211753612854E4C212F201B020537C2AFC2241204A175220075230075A913C6
:2012200075A71075C10075A700D3E55713F557C3E55A13F55AC3E55613F556E55DC560F5A6
:201240005DE55EC561F55EE55FC562F55F7563E1D2AF202517C3E5379404500612039002AC
:2012600010ADC2AF120435D2AF02102575370078A4E66006D290D292D294021048FFFFFFA6
:202FE000FFFFFFFFFFFFFFFFFFFFFFFFFFFFFFFFFFFFFFFFFFFFFFFFFFFFFFFFFF020ECC12
:203000000012CCFFFF010132FF093001FF55AAFFFFFFFFFFFF04FFFFFFFFFF285004FF02F3
:20302000FFFFFF07FFFFFF0000FFFFFFFFFFFFFFFFFFFFFFFFFFFFFFFFFFFFFFFFFFFFFFA6
:2030400023435F585F333023202020202020202023424C48454C492445464D38423531239C
:20306000426C75656A6179202020202020202020023A042034420D00452D0D0034420D007F
:203080004E27D300452DD01934190000000000000000000000000000000000000000000040
:2030A000000000000000000000000000000000000000000000000000000000000000000010
:2030C0000000000000000000000000000000000000000000000000000000000000000000F0
:2030E000000000000000000000000000000000000000FFFFFFFFFFFFFFFFFFFFFFFFFFFFDE
:10F00000C2AFC2D37597DE7597AD7581C075A90083
:10F0100075243875250331D87529A5752AF143F172
:10F020002053A4DFD28575D4FF75E3407DFA7803C1
:10F0300079E67C1075220075230090F1E57B06755A
:10F0400024987525013085020145208508D8FBD913
:10F05000F9DCF701B7308508D8FBD9F9DCF701B73F
:10F060003198E493A3C39A6004DDC301B7DBDB31BD
:10F070008A6002012E7B08E493FAA3316BDBF87AF5
:10F0800030316B752200752300318AEAFCEBFDC339
:10F09000ED94FE400E318A8A278B28ED30E0048AF9
:10F0A000828B83318A7AC270D8C3ED94FE60195086
:10F0B000CEBD0029EC600F7520007521FF75290079
:10F0C000752A000200000100A827A9280809D80411
:10F0D000D90201DA318EEAF201CE0D01A3C3ED941B
:10F0E000035051EDA2E092007AC5C3E5829400E599
:10F0F0008394F0508C200010438F02438F018529A8
:10F10000B7852AB7F0300027A827A9280809438F18
:10F1100001538FFDD804D902212FC3E58394F04019
:10F1200003A32114E28529B7852AB7F0A32114533C
:10F130008FFC017F7AC1BD030CE493A3FA314FDC4D
:10F14000F83147017F0181AA22AB23316BEBFAEA48
:10F150006222752608C3E52313F523E52213F52261
:10F1600050066323A0632201D526EA31D831D87531
:10F17000260AEAF4200102D285300102C28531D884
:10F18000C3134002C201D526EB22318EEAFB208553
:10F1900002218E3085022193752608AE24AF25C347
:10F1A000EF13FFEE13FE31DC31D8C3EA13308502D2
:10F1B0004480FA30E703632201C3E52313F523E516
:10F1C0002213F52250066323A0632201D526D9E538
:10F1D0002265236523F52222AE24AF250E0FDEFE25
:10F1E000DFFCD20122424C48656C6934373164E857
:03F1F000B5060160
:00000001FF
